:100000008A01172851285F28712884288F28A12861
:10001000D828820748346F346C34613420344D342E
:1000200075346E3464346F3421342134003402204A
:100030008A110A1207208A110A123C308312A60084
:1000400006208A110A120F308312A60006208A1198
:100050000A128312A40183122408A0000A3E003071
:100060000318013E8A0020080920003C031950288B
:10007000FA308312A10008208A110A128312240880
:10008000A0000A3E00300318013E8A002008092023
:100090008312A50004208A110A128312A40A2B28B5
:1000A000172883128501F8308316850006309F00DB
:1000B0008312051005118510831686010800FF3094
:1000C000831686008312851483120511000005151E
:1000D0000000861B64280511000085108316860128
:1000E00008008312851005102508860003208A1158
:1000F0000A12831205140515000005112D30A30006
:1001000005208A110A120800A30CA30C3F30A30596
:100110000330A3020000A30B8A280000080083120A
:10012000851005102608860003208A110A12831202
:100130000515000005112D30A30005208A110A12B3
:1001400008003C308312A60006208A110A120530EE
:100150008312A10008208A110A123C308312A600E3
:1001600006208A110A1205308312A10008208A1184
:100170000A123C308312A60006208A110A120530AA
:100180008312A10008208A110A1208308312A600E7
:1001900006208A110A1201308312A60006208A1155
:1001A0000A1206308312A60006208A110A120800DD
:1001B0008E308312A200000000000000000000004A
:1001C0000000A20BDD280000A10BD82800000800C9
:00000001FF
